:0200000480007A
:100000006F008004732F2034930F80006308FF0378
:10001000930F90006304FF03930FB0006300FF038E
:10002000130F000063040F0067000F00732F2034CC
:1000300063540F006F00400093E19153171F0000BD
:1000400023223FFC6FF09FFF93000000130100008C
:10005000930100001302000093020000130300004C
:100060009303000013040000930400001305000034
:10007000930500001306000093060000130700001C
:100080009307000013080000930800001309000004
:1000900093090000130A0000930A0000130B0000EC
:1000A000930B0000130C0000930C0000130D0000D4
:1000B000930D0000130E0000930E0000130F0000BC
:1000C000930F0000732540F16310050097020000B4
:1000D000938202017390523073500018970200000F
:1000E00093824202739052309B021000939252030B
:1000F0009382F2FF7390023B9302F0017390023AF5
:100100007350403097020000938242017390523046
:10011000735020307350303093010000970200007C
:10012000938282EE73905230130510001315F5017F
:10013000635C05000F00F00F930110009308D005D9
:10014000130500007300000093020000638A0200A0
:1001500073905210B7B200009B82921073902230BD
:100160007350003097020000938242017390123462
:10017000732540F17300203093000000130100004C
:1001800033B720009303000093012000631C774ED7
:10019000930010001301100033B7200093030000F8
:1001A000930130006310774E93003000130170000C
:1001B00033B7200093031000930140006314774C81
:1001C000930070001301300033B720009303000048
:1001D000930150006318774A930000003701020032
:1001E0001B01F1FF1311F10033B72000930310003E
:1001F00093016000631877489B0010009390F00112
:100200001301000033B72000930300009301700036
:10021000631A77469B0010009390F00137010200AB
:100220001B01F1FF1311F10033B7200093031000FD
:100230009301800063187744930000003781000029
:100240001B01F1FF33B720009303100093019000CE
:10025000631A7742B70000809B80F0FF1301000013
:1002600033B72000930300009301A000631C774084
:10027000B70000809B80F0FF378100001B01F1FF79
:1002800033B72000930300009301B000631C773E56
:100290009B0010009390F001378100001B01F1FFDB
:1002A00033B72000930300009301C000631C773C28
:1002B000B70000809B80F0FF370102001B01F1FFB7
:1002C0001311F10033B72000930310009301D00005
:1002D000631A773A930000001B011000131101020A
:1002E0001301F1FF33B72000930310009301E000E6
:1002F000631A77389B001000939000029380F0FF00
:100300001301100033B72000930300009301F000A5
:10031000631A77369B001000939000029380F0FFE1
:100320001B011000131101021301F1FF33B720006C
:100330009303000093010001631677349300E000FB
:100340001301D000B3B0200093030000930110010B
:10035000639A70329300B0001301D00033B12000D3
:100360009303100093012001631E71309300D000AD
:10037000B3B0100093030000930130016394703018
:10038000130200009300B0001301D00033B7200027
:10039000130307001302120093022000E31452FE1D
:1003A0009303100093014001631E732C130200009D
:1003B0009300E0001301D00033B7200013000000C9
:1003C000130307001302120093022000E31252FEEF
:1003D00093030000930150016316732A1302000077
:1003E0009300C0001301D00033B7200013000000B9
:1003F00013000000130307001302120093022000F1
:10040000E31052FE9303100093016001631C7326F6
:10041000130200009300E0001301D00033B7200066
:100420001302120093022000E31652FE9303000011
:100430009301700163187724130200009300B00049
:100440001301D0001300000033B720001302120084
:1004500093022000E31452FE9303100093018001E5
:1004600063127722130200009300F0001301D00002
:10047000130000001300000033B720001302120025
:1004800093022000E31252FE9303000093019001B7
:10049000631A771E130200009300A00013000000EF
:1004A0001301D00033B72000130212009302200082
:1004B000E31452FE930310009301A0016314771C10
:1004C0001302000093000001130000001301D0008C
:1004D0001300000033B72000130212009302200023
:1004E000E31252FE930300009301B001631C7718DE
:1004F000130200009300900013000000130000009E
:100500001301D00033B72000130212009302200021
:10051000E31252FE930310009301C0016314771697
:10052000130200001301D0009300100133B7200024
:100530001302120093022000E31652FE9303000000
:100540009301D00163107714130200001301D0004F
:10055000930080001300000033B720001302120044
:1005600093022000E31452FE930310009301E00174
:10057000631A7710130200001301D00093002001CA
:10058000130000001300000033B720001302120014
:1005900093022000E31252FE930300009301F00146
:1005A0006312770E130200001301D0001300000045
:1005B0009300700033B72000130212009302200052
:1005C000E31452FE9303100093010002631C770AA8
:1005D000130200001301D00013000000930030014B
:1005E0001300000033B72000130212009302200012
:1005F000E31252FE93030000930110026314770884
:10060000130200001301D0001300000013000000CB
:100610009300600033B72000130212009302200001
:10062000E31252FE9303100093012002631C77042F
:100630009300F0FF33311000930310009301300258
:10064000631271049300F0FF33B1000093030000C4
:100650009301400263187102B3300000930300005D
:100660009301500263907002930000011301E001B6
:1006700033B0200093030000930160026314700004
:10068000631030020F00F00F63800100939111009E
:1006900093E111009308D005138501007300000059
:1006A0000F00F00F930110009308D0051305000010
:0C06B00073000000731000C00000000088
:1010000000000000000000000000000000000000E0
:1010100000000000000000000000000000000000D0
:1010200000000000000000000000000000000000C0
:1010300000000000000000000000000000000000B0
:081040000000000000000000A8
:040000058000000077
:00000001FF
